:0300000002110BDF
:03000B000200A54B
:03002B000202AB23
:03005B0002045C40
:030073000204364E
:1000800002030406080C10182030406080040608A3
:100090000C10182030406080A0C00D0D0403060D28
:1000A0000502030202C2AFC0D0C0E020620C20688B
:1000B00002419A306602415AE47385258AC262E59C
:1000C00025F470022121206802210E758B00D0E0FA
:1000D000D0D0C293C295C297D2AF32C293C295C25A
:1000E00097740AD5E0FDE53C1420E21520E10D20CF
:1000F0007D02D296307D02D29202011ED29402017C
:100100001E207D02D292307D02D29602011E758B96
:1001100000D0E0D0D0C293C295C297D2AF32758BD7
:1001200000D0E0D0D0D2AF32419AE525600A207DE0
:1001300002D293307D02D297C295419AE5256002A2
:10014000D295207D02C297307D02C293419AE52567
:10015000600A207D02D297307D02D293207D02C2B8
:1001600093307D02C297419A207D02C292307D0277
:10017000C296207D02C296307D02C292740AD5E0FA
:10018000FDE525600A207D02D293307D02D297C220
:1001900095419A207D02C292307D02C296C294742B
:1001A0000AD5E0FDE525600A207D02D293307D026C
:1001B000D297C295419AC294207D02C292307D02AC
:1001C000C296740AD5E0FDE5256002D295207D0235
:1001D000C297307D02C293419AC294207D02C2969A
:1001E000307D02C292740AD5E0FDE5256002D29509
:1001F000207D02C297307D02C293419A207D02C2C7
:1002000096307D02C292C294740AD5E0FDE5256065
:100210000A207D02D297307D02D293207D02C293C4
:10022000307D02C297419A207D02C296307D02C283
:1002300092207D02C292307D02C296740AD5E0FD02
:10024000E525600A207D02D297307D02D293207D81
:1002500002C293307D02C297419A30723DE53C2044
:10026000E21A20E129207D02C292307D02C296204E
:100270007D02C296307D02C29202029A20E1E620FF
:100280007D02C292307D02C296C29402029AC2944A
:10029000207D02C296307D02C292E525F4F58A7572
:1002A0008B00D262D0E0D0D0D2AF32C2AFC2AD5359
:1002B000E6EFC0D0C0E0D2D3D2AFC2CEE52960070E
:1002C0002074461529610978007900E580307E01A7
:1002D000F430E30278FF53DACF207E0343DA203094
:1002E0007E0343DA10C2D8C271E580307E01F4305B
:1002F000E30279FFC3E89970CE306103752940208D
:1003000074037529408859D270E52A6004152A6162
:100310001920740543DA01C2D82070026141A8593E
:10032000206102C270207402612A882230690AC3E7
:10033000E522955E4003855E227882B6040385221D
:1003400024C3E52594404002D26420CF0CD0E0D0F5
:10035000D0C2D343E610D2AD32C2CF7802E52960D5
:10036000053074021529C3E55994014005755C00F8
:100370006183755D00756400E55C2401F55C5003E4
:10038000755CFF7982B7020EE547601EC3E52294D3
:100390003240178546227982B7030FE547600BC3C9
:1003A000E52294324004798E8722C3E523952260AA
:1003B000084004152361B90523D8C80564E56470B5
:1003C000021564D565647565017805C3E5649566B5
:1003D0004058C3E5649567500878017565030203CA
:1003E000EDC3E564956850057801756501C3E55F67
:1003F0009524401F7982B70402811FE54770148558
:10040000245FE56404600385666475650175233CBB
:1004100002042AE55F285005755FFF811FF55FE53F
:100420005F047006755DFF7564FFD0E0D0D0C2D365
:1004300043E610D2AD32C0D0C0E0C2AF53917F537B
:10044000E67FC260759100C3E49550F594E4955140
:10045000F595759104D0E0D0D0D2AF32C2AF53E65B
:10046000EFC2ADC0D0C0E0C0F0D2D3D2AFA8FBA9DC
:0E047000FCC2D830710281C353DACF207E0364
:10047E0043DA10307E0343DA20D271E580307E01FC
:10048E00F420E302819A88268927C19A53DACF2075
:10049E007E0343DA20307E0343DA10C2D8C27130B5
:1004AE007402C1867800E580307E01F430E302C12B
:1004BE00868859C16D53DACF207E0343DA20307E11
:1004CE000343DA10C271206102A19353DACF207E6A
:1004DE000343DA10307E0343DA20C2D8D271885437
:1004EE008955C3E89552F8E99553F9E4FB7E027AF3
:1004FE0000C3E8948CE994005005755800A183C39D
:10050E00E894C8E994005008E4D2E4FB7A0AA160AA
:10051E00C3E89468E994015008E4D2E3FB7A0FA192
:10052E0060C3E894D0E994025008E4D2E2FB7A1E4C
:10053E00A160C3E894A0E994055008E4D2E1FB7AE7
:10054E003CA160C3E89498E994085008E4D2E0FB1B
:10055E007A787E00C3E89556FCE99557FD30E7089A
:10056E00ECF42401FCEDF4FD755800C3EC9AED9EFD
:10057E00500375580188568957A854A95588528931
:10058E00537802C16DC3E89526F8E99527F9307CBA
:10059E0002C151307B02C151307A02C14A2075022C
:1005AE00A1B6E9FDE8FCA1D5E9C313F9E813F830CB
:1005BE007902C14AE9C313F9E813F8307802C14A47
:1005CE00E9C313FDE813FC206126C3EC941CED94E3
:1005DE00024002A1ECED7018C3EC94C8501205282D
:1005EE00C3E528940A5002C186755900D270C1869F
:1005FE00E528600215287400207F037896E624FA19
:10060E00FEE43400FFC3EC9EFCED9FFD5006780027
:10061E007900C151C3EC94FFED9400400678FF7948
:10062E0000C151EC856FF0A4C5F0A2F733F8790044
:10063E00400302066D78FF790002066DE9C313F9D7
:10064E00E813F8307C0EE9600278FFC3E81338F83F
:10065E00E43400F9C3E894FFE99400400278FF887F
:10066E0059D270206102C186741FF4552F4BF52F9D
:10067E00C274E42B7002D27475294030740375294C
:10068E000A306102C19A20740353DAFE752A2030B3
:10069E007403752A0AD0F0D0E0D0D0C2D3D2AD43C5
:1006AE00E6103279010206CF79030206CF790A02EB
:1006BE0006CF791E0206CF79640206CF79C80206EC
:1006CE00CF7817E4D5E0FDD8FAD9F6227A147B78E4
:1006DE000206F67A107B8C0206F67A0D7BB40206C1
:1006EE00F67A0B7BC80206F6AC257525017902B2A7
:1006FE007DE4C294D5E0FDE5256002D295D5E0FDFE
:10070E00C295D5E0FDD294D5E0FDE525600A207DA9
:10071E0002D293307D02D297E570D5E0FD207D02A6
:10072E00C293307D02C2977496D5E0FDD9C1EAF826
:10073E00D5E0FDD8FBDBB1C2948C2522C37C007DB5
:10074E000075F00005F0EA33FAEB33FB50F6EB13CD
:10075E00FBEA13FAC3E9FFE8FEE89AF8E99BF950C1
:10076E0004EFF9EEF8B3EC33FCED33FDD5F0DFED2D
:10077E00F9ECF822E889F08A20D2D4F8A9F07B00AF
:10078E0030F70B7BFFF42401F8E9F43400F9E88527
:10079E0020F0A4ADF0F8E98520F0A4AFF0FEED2E28
:1007AE00F974003FFA7C04C3EA13FAE913F9E8136B
:1007BE00F8DCF48BF030F70AE8F42401F8E9F434AD
:1007CE0000F9E889F0C2D4F8A9F0227882B60403C1
:1007DE0002087BC3E5599419401FE52D5406701984
:1007EE00E547703878057994E7146007780A146045
:1007FE00027812C3E53B984020E547600985615FAA
:10080E007564FF756501852224E4F53EF53FF540DC
:10081E00F541F542F54702087B7547017994E714D7
:10082E007013E523F43333F913F8E9540104F9E8AE
:10083E0054FE02086FE714147014E523F4333333B7
:10084E00F913F8E9540304F9E854FC020877E52398
:10085E00F433333333F913F8E954070404F9E85445
:0E086E00F8C39440F8E99400F9883E893F22CF
:10087C00E547603BC3E53B13F9E53A13F8C3E53EA6
:10088C0098F8E53F99F9500CC3E89480E994FF403F
:10089C00160208B7C3E8947FE9940050030208B726
:1008AC00787F79000208B7788079FF8843894422E1
:1008BC00E5476058E5432540F8E5443541F9854462
:1008CC0020E4300701F43542FA30E709C3EA94F02A
:1008DC0040150208F9C3EA940F50030208F978FF97
:1008EC0079FF7A0F0208F9780079007AF0C3E524D1
:1008FC00955E5006E52460092112E54420E70D21A0
:10090C0012E54430E706884089418A4222E5477067
:10091C000302097D78A1E6FAC3E54333F8E54433D5
:10092C00F9120782E930E70BC3E89480E994FF40A1
:10093C00132154C3E8947FE9940050022154787F2A
:10094C0079002154788079FFE820E715C3E52398D6
:10095C00F84009C3E89401400302097B78010209BD
:10096C007BE8F424012523F8400302097B78FF88F7
:10097C004522E54770030209E078A2E6FAA841A9EE
:10098C0042120782E930E70CC3E89401E994FF4076
:10099C00160209B7C3E894FFE9940050030209B7A3
:1009AC0078FF79000209B7780179FFE920E715C3D0
:1009BC00E54598F84009C3E8940140030209DE7844
:1009CC00000209DEE8F424012545F840030209DEA3
:1009DC0078FF88242278FFC264E52D5406702FD24C
:1009EC0064C3E53B940A4009C3E52594405002C218
:1009FC0064E53B601974FF853BF0848537F0A4F8FF
:100A0C00C5F0600278FFC3E895615002A861886068
:100A1C00227883E6F520120F2C75E8901206B1753A
:100A2C00E890E5E820ECFBA8BDA9BE120FAC756BF5
:100A3C0030756C00C3740013FD743013FC74302CCF
:100A4C00FC74003DFDECFAEDFBC3E89AE99B401405
:100A5C00E56B2430F56BE56C3400F56CEA2CFAEBA5
:100A6C003DFB80E5AE6BAF6CC3E56C13F9E56B1326
:100A7C00F8C3E913F9E813F8E56B28F569E56C3967
:100A8C00F56A7A03C3E913F9E813F8DAF7AA201A1E
:100A9C007009756B00756C00020AB71AEA6008EEF3
:100AAC0028FEEF39FFDAF88E6B8F6C2275E89022F6
:100ABC007883E6FFE5E820ECF7A8BDA9BE056DC379
:100ACC00E56D94084052756D00E9FA79A0E7604431
:100ADC00EA7007E56E601B020AF2C3E8956E6010BF
:100AEC00E56E5006600C14020AFE0460F9020AFE60
:100AFC00E56EF56EC394A8401B755EC0C3940540AB
:100B0C0013755E80C39405400B755E40C39405401D
:100B1C0003755E0075BB0122EFC39401601BC3E833
:100B2C0094FFE994035012C3E8956BE9956C500956
:100B3C00E55E600C155E020B4CE55EF46002055E32
:100B4C00A85EC3E524985002A824C3E8955F400A28
:100B5C00A85FE55FF46003855F5E8825E56DB407EB
:100B6C000375BB1E22743279A387F0A4C5F0A2F7DB
:100B7C0033F8C3E8955E4002A85E88228824882555
:100B8C00886122753A00753B7F2275C820A8CCA9D4
:100B9C00CD75C824AA38AB3988388939C3E89AF896
:100BAC00E99BF9AA3AAB3BAC3AAD3B7E047F02C35E
:100BBC00EB940440021E1FC3EB940840021E1FC39B
:100BCC00ED13FDEC13FCDEF7C3EA9CFAEB9DFBEF97
:100BDC006009C3E913F9E813F8DFF7EA28FAEB39EF
:100BEC00FB8A3A8B3B400122753AFF753BFF223062
:100BFC00600261FB854C50854D51D26043E68022EA
:100C0C007892E6FFC3E535948240010FC3E5359435
:100C1C00A040010FC3EF940640027F057E021E30F8
:100C2C0072010EC3E53B940350060E0E3072010E9A
:100C3C00C3E53B940250060E0E3072010EA93BA880
:100C4C003A7A04C3E913F9E813F8DAF7C3E89EF823
:100C5C00E99400F94009C3E89402E994005004783F
:0E0C6C0002E4F9E9FBE8FAC3E913FDE813FC22
:100C7A00884C894DC3EF94036037EF20E00DE82CD0
:100C8A00F8E93DF9ECFAEDFB020CA8E828F8E93995
:100C9A00F9C3E89402F8E99400F97A02E4FBC3EF95
:100CAA009403400D8A4E8B4F884889498C4A8D4B54
:100CBA0022884E894F8A488B498C4A8D4B22306054
:100CCA000281C8D26043E680E52D54066027A83A1F
:100CDA00A93BE53494085006E820E002A94D759135
:100CEA0000C3E498F594E499F595759104D260539C
:100CFA00917F43E68022D265753D00752000020D82
:100D0A0013D265753D00752040E52D54066002C278
:100D1A0065D2AF206005E53D60012278017A02C301
:100D2A00E53B940540027802C3E53B940A40027809
:100D3A0003C3E53B940F40027A03306904781E7AB4
:100D4A0001206007E53D6003D2AF22D2AF0000C2A6
:100D5A00AFC3E53BFB940F40027B0FEB04307301FA
:100D6A002320620123F93069027982E58BC3994015
:100D7A00D0053DEAFBE59E7005E59B020D8AE59AE2
:100D8A005440B52004DBEEA1B7206502A113C26569
:100D9A00759100AE3AAF3BC3E49EF594E49FF59596
:100DAA00759104D26053917F43E680A113306502A6
:100DBA00A113D88DD2AF2230690B05342060167585
:100DCA003400020DDF20600D20650A206B071581B3
:100DDA0015810215DF22A84EA94F75910053917F04
:100DEA00C3E498F594E499F595759104854850857E
:100DFA004951D26043E680227800306405306502AA
:100E0A007801E53575F007A4F9E5F028F5F0E9A2CF
:100E1A00F013A2F113A2F213F535C39478500375B7
:100E2A003578C3E53595364008D266C293C295C275
:100E3A0097306002C13B854A50854B51D26043E6E8
:100E4A008022C2AFC292C294C29630720B9001FC49
:100E5A00740AD5E0FD020E62207D02D292307D0234
:100E6A00D296759F33759E00753C02020FA7C2AFDA
:100E7A00207D02C297307D02C2933072179001D949
:100E8A00C294207D02C296307D02C292740AD5E0D5
:100E9A00FD020EA190013C306206E5256002D29562
:100EAA00207D03759E23307D03759E22753C0302C7
:100EBA000FA7C2AFC292C294C29630720B9001B60B
:100ECA00740AD5E0FD020ED2207D02D296307D0250
:100EDA00D292207D03759E22307D03759E23753C38
:100EEA0004020FA7C2AFC295307217900193207DFA
:100EFA0002C292307D02C296C294740AD5E0FD0203
:100F0A000F0F90012A30620EE525600A207D02D279
:100F1A0093307D02D297759F33759E00753C05020A
:100F2A000FA7C2AFC292C294C29630720B900168E8
:100F3A00740AD5E0FD020F42D294207D03759E23E8
:100F4A00307D03759E22753C06020FA7C2AF207D35
:100F5A0002C293307D02C29730721F900227207D11
:100F6A0002C292307D02C296207D02C296307D0274
:100F7A00C292740AD5E0FD020F8790014E30620ECC
:100F8A00E525600A207D02D297307D02D293207D2A
:100F9A0003759E22307D03759E23753C01C266D27D
:100FAA00AF22900128C293C295C297C292C294C23C
:100FBA0096C2622278807607087607087601087654
:100FCA00040876FF0876FF08760708760208760195
:100FDA00087601788C76010876000876B40876FFE0
:100FEA000876FF0876FF0876030876FF0876010878
:100FFA0076FF0876250876D00876780876C80876C7
:10100A00040876FF08760108760008767A087610D2
:10101A00087601227887E6FFC2727888C27DE630B8
:10102A00E102D27DC27E7889E630E102D27EC3EF48
:10103A0094026008758E01D27302104B758E00C23D
:10104A0073227880E6149000809378A1F67881E67E
:10105A00149000809378A2F6120FAC227886E614D8
:0F106A0090008D9378A3F6120FAC22789FE6F8D2
:10107900700108C3E8941140027811E82828F56640
:101089002566256628F56725662828F56822789C4F
:10109900E67536FF75370CB402067536A075370A42
:1010A900B4030675368275370522227896E6FA78F2
:1010B90097E6FB307F047A007BFFC3EB9AFCC3946D
:1010C9008250027C82756F00056FEC856FF0A4C3B6
:1010D900E5F0948040F222D27F11B41206C07A0062
:1010E9007B007C101206B6E5592AFA74003BFBDC3A
:1010F900F37C04C3EB13FBEA13FADCF7FEC27F119E
:10110900B422E5EF20E6037520000520903DFFE5B8
:1011190020146006901FFF1460009304600375EFAC
:1011290012C2D353D9BF7581C043FF801206B1756E
:10113900EF0243B203E5B3240420E702F5B3120F2B
:10114900AC7580FF75A40075F1FE75D4F775900232
:1011590075A5FC75F2FC75D50075A0FD75A602751F
:10116900F30275D60075B0FF75A70175F4FF75E236
:1011790041120FBE12161A78988670C2AF1206CAAB
:101189001206DA1206C01206E11206C01206E812A9
:1011990006C012173D1206CA1206CA1206C5C2AF08
:1011A900E4F8F6D8FD78C879C8308307D9FBD8F7B1
:1011B900021C00120FBE12161A111E114C116611D3
:1011C90075119711B311B478988670120FAC7588A0
:1011D9005075891275C82475910475D84075A8226F
:1011E90075B80275E690759B80759D00759A807536
:1011F9009C0075D10E75BC5875BB0175BA1F75E891
:10120900801206B1D2AF120A1D43DA01C2D8C271E7
:101219001206CA753001D2617B037A0CE558700653
:101229007A0CDB0221A71206C020700221A7C27026
:10123900E559C3940240E3E52F541F855B5AF55BDA
:10124900B55AD7DAD7C26153DACF207E0343DA2001
:10125900307E0343DA10C2D8C271C27575280012F4
:1012690006C5307409C3E528940A4002D2751206EE
:10127900B678023074027800C3E5599840F0C2AFDD
:101289001206DA1206DA1206DAD2AF1206CA754661
:10129900001206B6788CE6C39401500302136EE57A
:1012A90030C39401500302136E207435C3E5599479
:1012B900FF500302136EC2AF1206EFD2AF1206C57A
:1012C900C3E559940150EFC2AF1206DA1206BB12F8
:1012D90006DAD2AF1206C5C3E55994FF40E90217F1
:1012E900C27F05D27F11B41206C5C2AFC27F11B445
:1012F900AE59C3E559947FD2AF40741206B1C2AF5B
:101309001206EFD2AFDFDC11E0C3EE94057897F651
:101319001206CA12165C1217457F0AD27F11B4123F
:1013290006C5C2AFC27F11B4AE59C3E559947FD285
:10133900AF50E61206B1C2AF1206DA1206BB1206A8
:10134900DAD2AFDFD611E0EE24057896F61206CA96
:1013590012165C1217741206C511B4C3E55994FF2D
:1013690040F40217C2C3E559954640038559461210
:1013790006C578017988E7B403027805C3E5599869
:101389004002419AC2AF1206EF1206EF1206EFD2DF
:10139900AF1206CA753000E4F531F5320531E53191
:1013A900F470390532789AE6781914601278321493
:1013B900600D787D14600878FA146003753200C3F3
:1013C900E53298401715327531B478998670C2AFF5
:1013D9001206EFD2AF789886701206C51206BBE5E1
:1013E90029700530740221A778012074027806C398
:1013F900E5599840A71206C5E529700221A7C2AF91
:10140900120FACE4F522F523F524F525D2AF788542
:101419008662F53EF53FF540F541F542F56DF54734
:10142900F52CF52DF535120B8F756D0875BB1E1250
:1014390006B1120AB8E5E820ECFBA8BDA9BEE9701F
:1014490001F8886E120ABC756D0875BB1E7887E6AF
:10145900FE7602111E7887EEF6C2AF755EFF120B9B
:0F1469007185225E85225F852260D2AF752201D8
:10147800752401752501855D64756501D268D26999
:10148800753400120F2C120F56120B8F120B961276
:101498000C0C0214A8120FAC111E756D0075BB015F
:1014A800120D0B120DC1120DE01207D9120E021205
:1014B8000E4C120B96120BFB120C0C120CC8120DD0
:1014C80000120DC1120DE012087C1209E1120E0281
:1014D800120E78120B96120BFB120C0C120CC8127F
:1014E8000D0B120DC1120DE01208BC120E02120EE5
:1014F800BC120B96120BFB120C0C120CC8120D002E
:10150800120DC1120DE0120919120E02120EEE127E
:101518000B96120BFB120C0C120CC8120D0B120DB1
:10152800C1120DE012097E120E02120F2C120B9638
:10153800120BFB120C0C120CC8120D00120AB81276
:101548000DC1120DE0120ABC120E02120F56120B38
:1015580096120BFB120C0C120CC830692F206B2C46
:1015680085615E85615F855D6475650179327A0A9A
:10157800C3E534994009C269D26A8A33021594C313
:10158800E559940140030214A80215DF306A1B20B4
:101598006B18E533147004C26A819DF533C3E559AD
:1015A800940140030214A80215DFC3E55C940140CE
:1015B8000985615F855D64756501C3E55C94FA50D2
:1015C80016307404E529600FC3E53B78F0306B02F0
:1015D800786098500281A8C2AF120FAC7887E6FEF7
:1015E8007602111E7887EEF6E4F522F523F524F548
:1015F80025F562C268D2AF1206B1120FAC3074067C
:10160800E529700221A7788DE6C39401400241774D
:1016180061A0901A0D782012169EE520B4A50CA39F
:1016280012169EE520B45A0302163C120FBE12167B
:101638005C02165B901A0378807B0A12169EA30838
:10164800DBF9901A0F788C7B1512169EA308DBF92C
:10165800901A2422C2AF1216DD1216B7901A00741F
:101668000D1216A3A374021216A3A374131216A3C1
:10167800901A0378807B0A1216A2A308DBF9901A45
:101688000F788C7B151216A2A308DBF91216F0123C
:1016980016CE901A2422E493F622E6438F01538F44
:1016A800FD75EF0275B7A575B7F1F0538FFE2243AC
:1016B8008F02438F0175EF0275B7A575B7F1901AC0
:1016C8000DF0538FFC22901A0D74A5D1A3901A0E19
:1016D800745AD1A3227A3079D07820901A40D19EBA
:1016E800E520F709A3DAF7227A3079D0901A40E793
:1016F800D1A309A3DAF922AB71A872BB01027980E0
:10170800BB02027981BB03027982BB04027994BBD4
:1017180005027983BB06027986BB07027992BB086A
:10172800027987BB0902799CBB0A027988BB0B0244
:101738007989E8F7227C051206CADCFB22C2AF12BF
:1017480006DA1206E11206E81206EF1206BB1206C6
:10175800DA1206E11206E81206EF1206BB1206DAE2
:101768001206E11206E81206EFD2AF22C2AF120645
:10177800EF1206E81206E11206DA1206BB1206EFAD
:101788001206E81206E11206DA1206BB1206EF127A
:1017980006E81206E11206DAD2AF22AE71AF72C2C3
:1017A800AF1206DA1206DA1206DA1206BBDEF212F7
:1017B80006EF1206BBDFF8D2AF22F145F13DF13D4D
:1017C800757101757201757300F1A37C05AD59122D
:1017D80006CAC3ED955970F5C3E5599401400AC38B
:1017E800E55994FF40330217FED1FFD15CF145C2A1
:1017F800AF75EF12F13DDCD50573C3E57394035063
:101808000280C612173D0572E5711490009A93F88C
:1018180008C3E57298500280AD12173D12173D05B6
:1018280071C3E571940C50028099120FBE12165CB8
:08183800C2AF75EF1212173D5B
:101A00000D021307070104FFFF07020101A55A0198
:101A100000B4FFFFFF03FF01FF25D078C804FF01DA
:051A200000FF1001FFB2
:101A4000235467794B4631323041485623202020B9
:101A500023424C48454C4923463331302320202033
:101A60002020202020202020202020202020202076
:101C0000C2AFC2D353D9BF7581C043B20343FF8073
:101C1000752438752503B1BF75EF0275E24043F1B5
:101C20000853A4F7D283780379E67C1075220075F7
:101C30002300901DCC7B0675249875250130830206
:101C4000813D208308D8FBD9F9DCF781AD308308CA
:101C5000D8FBD9F9DCF781ADB17FE493A3C39A60D7
:101C6000028126DBDDB171600281267B08E493FAF4
:101C7000A3B152DBF87A30B152752200752300B15E
:101C800071EAFCEBFDC3ED94FE400EB1718A278B27
:101C900028ED30E0048A828B83B1717AC270D8C398
:101CA000ED94FE601050CEBD0022EC600675200061
:101CB0000200008100A827A9280809D804D90281B8
:101CC000C9B175EA89AAF281BB0D8199C3ED94036C
:101CD0005049EDA2E092007AC5C3E5829400E58305
:101CE000941C5093200010438F02438F0175B7A5B9
:101CF00075B7F1F030001FA827A9280809438F0104
:101D0000538FFDD804D902A11689AAE275B7A5752B
:101D1000B7F1F0A3A103538FFC81757AC1BD030C09
:101D2000E493A3FAB136DCF8B12E81758177AA224B
:101D3000AB23B152EBFAEA6222752608C3E52313FE
:101D4000F523E52213F52250066323A0632201D573
:101D500026EAB1BFB1BF75260AEAF4200102D28398
:101D6000300102C283B1BFC3134002C201D526EBCA
:101D700022B175EAFB208302A175308302A17A7536
:101D80002608AE24AF25C3EF13FFEE13FEB1C3B197
:101D9000BFC3EA133083024480FA30E703632201B1
:101DA000C3E52313F523E52213F52250066323A090
:101DB000632201D526D9E52265236523F52222AECB
:101DC00024AF250E0FDEFEDFFCD20122424C486517
:0A1DD0006C6934373132F31006015C
:00000001FF
